:100000000C9446000C9463000C9463000C94630001
:100010000C9463000C9463000C9463000C946300D4
:100020000C9463000C9463000C9463000C946300C4
:100030000C9463000C9463000C9463000C946300B4
:100040000C9463000C9463000C9463000C946300A4
:100050000C9463000C9463000C9463000C94630094
:100060000C9463000C9463000C9463000C94630084
:100070000C9463000C9463000C9463000C94630074
:100080000C9463000C9463000C94630011241FBE55
:10009000CFEFD0E1DEBFCDBF11E0A0E0B1E0EAE4F8
:1000A000F2E000E00BBF02C007900D92A030B10754
:1000B000D9F711E0A0E0B1E001C01D92A030B10776
:1000C000E1F70C9465000C940000CDEFD0E1DEBFA9
:1000D000CDBF80E28093370082E880934F008AE1B1
:1000E00080934E0080E49CE9909347008093460003
:1000F00080914A0090914B0080914A0090914B0072
:100100002BE0893B920798F080914A0090914B0038
:1001100028E08939920780F380914A0090914B0042
:100120008456904090934B0080934A00EDCF88E92D
:1001300098E090934B0080934A001A82198289813B
:100140009A8123E18838920744F40E94040189814E
:100150009A8101969A838983F2CF80914A00909187
:100160004B0080914A0090914B002BE0883B920716
:1001700098F480914A0090914B002FE0803A9207CA
:1001800080F780914A0090914B008C599F4F90933B
:100190004B0080934A00EDCF1A82198289819A819F
:1001A00023E1883892070CF0A3CF0E9404018981D3
:1001B0009A8101969A838983F1CFCF93DF93CDB74C
:1001C000DEB780ED97E090934B0080934A00DF917B
:1001D000CF910895CF93DF93CDB7DEB788EB9BE047
:1001E00090934B0080934A00DF91CF910895CF9375
:1001F000DF93CDB7DEB780EA9FE090934B0080930A
:100200004A00DF91CF910895CF93DF93CDB7DEB74A
:1002100022970FB6F894DEBF0FBECDBF1A821982A7
:1002200089819A8123E18838920734F489819A81FF
:1002300001969A838983F4CF22960FB6F894DEBF95
:0A0240000FBECDBFDF91CF910895EE
:00000001FF
